:020000040000FA
:02000000802856
:080008008312692069208101C7
:100010000B11A00A0F302002031D54288312860AF8
:10002000A001A10AC730D420303021076E20E02083
:100030000A302102031D5428A101A20AC630D4208F
:10004000303022077720E02006302202031D54289A
:10005000A201A30AC430D420303023076E20E02050
:100060000A302302031D5428A301A40AC330D4205C
:10007000303024077720E02006302402031D542866
:10008000A401A50AC130D420303025076E20E0201D
:100090000A302502031D5428A501A60AC030D42029
:1000A00030302607E02054288B160900A001A1015A
:1000B000A201A301A401A501A601080004302502A4
:1000C000031DA12802302602031DA1285620A320CB
:1000D0000800BB30A800A80B6B280800A7003A3026
:1000E0002702031D75283030080027080800A700E4
:1000F00036302702031D7E2830300800270808000C
:1001000007309F0083169F01003086008500831210
:100110003830D4200130D4200330D4200F30D42004
:100120008030D420C030D420FF20A3200730831695
:100130008100831205108601003081008B178B1619
:1001400086015E20A128C730D42030302107E0206E
:10015000C630D42030302207E020C530D4203A30D9
:10016000E020C430D42030302307E020C330D42036
:1001700030302407E020C230D4203A30E020C130B3
:10018000D42030302507E020C030D420303026077E
:10019000E0208030D4205430E0204930E0204D3041
:1001A000E0204530E02008008600EC200430850087
:1001B000EC2000308500EC2004308500EC200800A5
:1001C0008600EC2006308500EC2002308500EC2013
:1001D00006308500EC2008001930AA00A900A90B00
:1001E000EF28AA0BEE280800FA30AA00A900A90BF4
:1001F000F728AA0BF6280800F420F420F420803019
:10020000D4205330E0204530E0205430E0203A3014
:10021000E020C030D4200630B70026308400033000
:100220008A008316F030860081138312EF30B0000D
:1002300086000430B100B00C30088600EC200608BF
:100240000F38B200B209031D2829B10B1B2916294A
:1002500006080F38B600B609031D2829831600309A
:1002600086008312B00930080F39B0003208F03927
:10027000B004300886001130B200B2033208002307
:100280003002031D3D29320886001030320700235A
:100290008600B000003083160030860083123008DC
:1002A000D03E8000303EE0208403B70B0F290800C9
:10060000820711341234143418342134223424343F
:10061000283441344234443448348134823484347C
:10062000883430343134323433343434353436343D
:100630003734383439344134423443344434453423
:0206400046343E
:02400E00293F48
:00000001FF
